:100000000C94BB010C94F3010C94F3010C94F301D8
:100010000C94F3010C94F3010C94F3010C94F30190
:100020000C94F3010C94F3010C94EE1D0C94C01E7F
:100030000C94CD180C94F3010C94F3010C94F3017F
:100040000C94F3010C94F3010C94F3010C94F30160
:100050000C94F3010C9455190C94F3010C94F301D6
:100060000C94F3010C9413160C94F3010C94F3010B
:100070000C94F3010C94F3010C94F3010C94F30130
:100080000C94F3010C94F3010C94F3010C94F30120
:100090000C94F3010C94F3010C94F3010C94F30110
:1000A0000C94F3010C94F3010C94F30115021D025E
:1000B00027022E0233023B025E02A404A404D004F1
:1000C000D004380556056E066E066105FA050B0666
:1000D0000B062D1F541F4C20541F4C20A01FC31F64
:1000E0004C201A2029200000E700000048004700AB
:1000F000460029003A006800E3008C008B008A006B
:100100002B0029003B006900E000E100E100E00075
:1001100014001E003C006A00E2001D0016000400EE
:100120001A001F003D006B0006001B0007000800BE
:10013000210020003E006C002C001900090017006F
:10014000150022003F006D00110005000B000A00A1
:100150001C00230040006E00E30010000D0018009A
:100160002400250041006F0036000E000C00120034
:100170002700260042007000370038000F003300CF
:1001800013002D00430071000000340031002F00E7
:100190002E00440072003500E50028003000000009
:1001A00000004500730051005000880052004C00D0
:1001B0004D002A004900000059004F005C005F001C
:1001C0004E004A004B00620063005A005D005E0072
:1001D000600053005400000058005B008500570089
:1001E000610055000000000000000000650056009E
:1001F0000000000000002C03490042004D002000D8
:100200005400650072006D0069006E0061006C00B2
:1002100020004B006500790062006F0061007200F1
:1002200064000000080351004D004B00000004036F
:10023000090409023B00020100A0FA0904000001C0
:10024000030101000921110100012240000705817D
:100250000308000109040100010300000009211145
:1002600001000122B60007058203200001120100EF
:100270000200000008EDFE356500010102000105E5
:10028000010902A10185020901A10005091901293D
:10029000081500250195087501810205010930093D
:1002A000311581257F95027508810609381581254C
:1002B0007F950175088106050C0A38021581257F96
:1002C000950175088106C0C005010980A10185035B
:1002D00019012AB700150126B70095017510810094
:1002E000C0050C0901A101850419012AA00215010C
:1002F00026A002950175108100C005010906A10123
:100300008506050719E029E71500250195087501FF
:1003100081020507190029EF1500250195F07501E7
:1003200081020508190129059505750191029501BC
:1003300075039101C005010906A101050719E0290E
:10034000E715002501950875018102950175088161
:10035000010507190029FF150026FF0095067508FD
:10036000810005081901290595057501910295017E
:1003700075039101C00011241FBECFEFDAE0DEBF8C
:10038000CDBF04B603FE18C08091F9029091FA0225
:10039000A091FB02B091FC028730904BA740B04B7C
:1003A00059F41092F9021092FA021092FB02109284
:1003B000FC02E0E0F8E3099511E0A0E0B1E0EEEF27
:1003C000F1E402C005900D92AC37B107D9F722E0F5
:1003D000ACE7B1E001C01D92A93FB207E1F70E946E
:1003E000EA100C94FD200C94000008958091840282
:1003F0008160809384020E940615EFE7F1E011927C
:1004000081E0E039F807D9F70C94F5010E94011654
:10041000E0917E014E2F50E04730510508F06FC04B
:10042000FA01EA5AFF4F0C9494208FEF0E942E1588
:100430008A3F09F064C081E00EC08A3A11F482E07C
:100440000AC0882309F45BC010927E0158C088233B
:1004500009F455C083E080937E0151C0882309F4DC
:100460004EC084E0F8CF88EF0E942E158A3F09F035
:1004700046C085E0F0CF882309F441C0803F11F4E5
:1004800086E0E9CF8838A8F7E82FE695E695E69567
:10049000F0E0E158FE4F4081877021E030E0B90183
:1004A00002C0660F771F8A95E2F7CB01242F30E058
:1004B00026233723232BE9F6842B1FC08823F9F04A
:1004C0008838B8F6E82FE695E695E695F0E0E1582D
:1004D000FE4F4081877021E030E0B90102C0660F15
:1004E000771F8A95E2F7CB01242F30E026233723AC
:1004F000232B09F4BECF809584238083BACF81E07B
:100500000895E82FF0E0E158FE4F808108950895A6
:10051000982F82FB882780F990FD826091FD84608E
:100520000C944A1681E0089581E008950C94940299
:1005300008950C9498021F93CF93DF9300D000D0BE
:100540001F92CDB7DEB749835A836B8330919101F7
:1005500089819A81311114C0662359F0222349F010
:100560000E94AB08182F682F89819A810E94540835
:1005700003C00E947F08182F69817A81812F04C0EF
:100580000E94AB0869817A810F900F900F900F90B5
:100590000F90DF91CF911F910C94C60FFC01262F75
:1005A000408151816281738184810C949B0281E03E
:1005B0000895CF93DF93EC0160E00E94CE02BE016C
:1005C000DF91CF910C94990208950E94FE060E943B
:1005D000E4022FEF84E39CE0215080409040E1F75B
:1005E00000C000000C947B190F931F93CF93DF93EF
:1005F0008C0161E00E94CE02EC01B8010E949602DB
:100600008823F1F1B801CE010E9419178823C1F1A6
:10061000B801CE010E948013882391F1B801CE0168
:100620000E947516882361F1F8018281882309F1FF
:10063000CB358DE5D807C1F050F4C115FCE5DF07D7
:1006400081F0CF3DDC45A9F40E94DC0D19C0CC350A
:10065000EDE5DE0761F0CD35DD4559F40E94250D4D
:1006600008C00E94E5020CC00E942E0D02C00E942C
:10067000310DC801DF91CF911F910F910C9492021F
:1006800080E0DF91CF911F910F9108950E94B018E3
:100690000C944F030E9452030C94B618089580E006
:1006A0000C9488020E9475170C9488020E9475179A
:1006B00090919001891721F0809390010C94880209
:1006C0000895CF93DF93CDB7DEB72B970FB6F8948D
:1006D000DEBF0FBECDBF4F83588769877A878B8770
:1006E00061110E94710C9E012F5F3F4F86E0F9015E
:1006F00011928A95E9F785E0FE013796D9010190BC
:100700000D928A95E1F789819A814C815D81452B13
:1007100031F09F3F31F491E08F3F19F403C091E035
:1007200001C090E090FF09C049815A816B817C81B2
:100730008D819E810E94920B05C0C9010E94D70243
:100740008111F2CF2B960FB6F894DEBF0FBECDBF4E
:10075000DF91CF910895FC01808191810E94ED0885
:100760000895CF93882309F450C0C82F8CEF8C0FC5
:10077000813AD0F46C2F80910201909103010E9484
:10078000EB17882349F06C2F8091020190910301AF
:100790000E9476180E94930C6C2F80910201909118
:1007A00003010E946B180CC080E28C0F883058F453
:1007B000C77081E001C0880FCA95EAF70E94540C07
:1007C000CF910C94930CEBE5EC0FE33040F4F0E0A8
:1007D000E95BFE4F808190E0CF910C94A917E8E58A
:1007E000EC0FE73150F4F0E0EE0FFF1FE75EFE4F35
:1007F00080819181CF910C94BF17CD3E30F08C2F2A
:100800000E946F11CF910C944112CF9108958823CB
:1008100089F19CEF980F913A40F4682F8091020182
:10082000909103010E9476180DC090E2980F9830C5
:1008300058F4877091E001C0990F8A95EAF7892FE3
:100840000E945A0C0C94930C9BE5980F933020F463
:1008500080E090E00C94A91798E5980F973120F468
:1008600080E090E00C94BF178D3E20F00E94CA11EA
:100870000C94411208951F93CF93DF93182FEB012F
:100880000E94B103209741F08FE99FE00197F1F7B3
:1008900000C000002197F6CF812FDF91CF911F91EB
:1008A0000C940704893319F060E070E002C060E541
:1008B00070E00C943B04882321F00E94540C0C94AB
:1008C000930C0895882321F00E945A0C0C94930CE9
:1008D0000895CF92DF92EF92FF920F931F93CF93E1
:1008E000DF937C01D62FC72FFC0112810581029571
:1008F0000F700E944A0C8823B9F01123A9F08C2FA5
:10090000807F803421F080E28D0F883068F0809104
:10091000E70282FD09C082E00E94F30C0E944A0CAB
:1009200091E0D82ED92601C0D12CCC2EC2948FE0D4
:10093000C8228C2D90E08C30910508F0CFC1FC01CD
:10094000E35AFF4F0C9494208C2F807FCF70882324
:1009500011F0C295C07F112399F0CC2309F4AAC1EC
:1009600080E28D0F883010F0D11104C08C2F0E94CE
:10097000540C03C08C2F0E94640C0E94930C9AC1EB
:100980008D2F0E940704CC2309F4A8C180E28D0FAB
:10099000883038F1DD2329F18C2F0E946A0C24C0A5
:1009A0008C2F807FCF70803211F0C295C07FDD2305
:1009B00019F0D130A1F13DC08091E70282FF17C04C
:1009C000112349F0CC2329F08C2F0E94540C0E9453
:1009D000930C80E070C180E00E940704CC2309F4EE
:1009E0007DC18C2F0E945A0C0E94930C77C1112359
:1009F00071F0002341F0013031F40E94740C8C2B13
:100A00000E947C0C6BC10E94740C8C2B1DC00023B7
:100A100019F0013009F462C10E94890C25C011232C
:100A200021F0063008F05AC10EC0053008F056C15A
:100A30001BC0112361F0002331F0F701858180FF95
:100A400039C18F7085838C2F0E945B0447C10023BE
:100A500059F0D93309F03FC1FFEF07EE13E0F15031
:100A600000401040E1F735C18C2F0E94620436C16E
:100A70008C2F86958695837019F0813061F02EC198
:100A8000112321F08D2F9C2F937002C080E090E005
:100A90000E94A9172BC1112321F08D2F9C2F937039
:100AA00002C080E090E00E94BF1720C18D2F11236B
:100AB00019F00E946F1102C00E94CA110E944112D7
:100AC00015C18C2F837009F047C011110BC12D2F58
:100AD000229526952770220F220F6D2F6F70862F7B
:100AE00090E0A0E0B0E0022E04C0880F991FAA1F7A
:100AF000BB1F0A94D2F7D4FF10C04FE050E060E073
:100B000070E004C0440F551F661F771F2A95D2F767
:100B1000409550956095709503C040E050E0BA0153
:100B2000C695C695C3708A019B01082B192B2A2BE9
:100B30003B2BC901B801C23049F058F4C13019F05B
:100B40000E946A07CFC00E945807CCC00E947C0751
:100B5000C9C00E945607C6C0112319F08C2F81709E
:100B600001C08695882309F4BDC02D2F22952695B6
:100B70002770220F220F6D2F6F70862F90E0A0E05C
:100B8000B0E0022E04C0880F991FAA1FBB1F0A9451
:100B9000D2F7D4FF10C04FE050E060E070E004C036
:100BA000440F551F661F771F2A95D2F74095509521
:100BB0006095709503C040E050E0BA01C695C695B7
:100BC000C3708A019B01082B192B2A2B3B2BC901CF
:100BD000B801C23049F058F4C13019F00E942F0812
:100BE00081C00E941D087EC00E9441087BC00E94F7
:100BF000900778C0CF70112339F08C2F0E94B60770
:100C00008D2F0E945B046EC08D2F0E9462048C2F7A
:100C10000E94D70767C0D23F21F128F4D03F41F0AE
:100C2000D13FC1F043C0D33F19F1D43F79F03EC06A
:100C3000112341F0053008F051C08C2F8F710E94B4
:100C4000FC074CC0063008F049C0F7CF8091E7029E
:100C500082FF18C0112339F08C2F8F710E94B607C4
:100C60003DC01123C9F38C2F8F710E94D70736C066
:100C7000112329F08C2F8F710E94A1072FC00E9491
:100C80009C072CC0112349F0CF718C2F0E94B6070E
:100C900063E08C2F0E94D80C21C081E00E94F30CED
:100CA0000230E0F082E00E94F30C18C0112331F012
:100CB000002391F28D2F0E94B10310C0002399F2FE
:100CC000D93349F41FEF27EE33E011502040304074
:100CD000E1F700C000008D2F0E94070488EF8C0D03
:100CE000843020F40E9475170E948802DD20C9F02C
:100CF0000E94460C80FD15C0F70112820E94400C34
:100D00000E94B607C7010E94B2060E94400CDF9104
:100D1000CF911F910F91FF90EF90DF90CF900C94A7
:100D2000D707DF91CF911F910F91FF90EF90DF9048
:100D3000CF9008950F931F93CF93DF93EC016881B9
:100D400079818A810E94F8088C010E9453080E94D0
:100D50004407B801CE010E946904DF91CF911F9131
:100D60000F910895CF93DF93EC01988189812B81B6
:100D70003C81232B31F08F3F31F481E09F3F19F408
:100D800003C081E001C080E080FD1DC0CE010E9453
:100D9000F402811110C00E944A0C8823A1F08A81BC
:100DA000882389F08091E70282FD0DC082E0DF9107
:100DB000CF910C94F30CCE010E949A06CE01DF91E4
:100DC000CF910C94D902DF91CF91089580E090E00B
:100DD0000E94A91780E090E00E94BF170E94710C4A
:100DE0000E94930C0E9472130C9441128091020194
:100DF000909103010E9481180C94E6060E94610CF8
:100E00000C94F60692959F70963079F010F49250FB
:100E100001C09A50923068F4803F69F018F4883E1F
:100E200040F409C0843F29F406C0883E20F0813F89
:100E300011F080E0089581E00895FC0180819181A6
:100E40000E94ED080E9402070895CF93DF9300D01F
:100E500000D01F92CDB7DEB70F900F900F900F907C
:100E60000F90DF91CF910895CF93DF9300D000D002
:100E700000D0CDB7DEB726960FB6F894DEBF0FBE12
:100E8000CDBFDF91CF910895089508950C94450743
:100E90000C9446070E9448076093EB017093EC01A5
:100EA0008093ED019093EE010C94E6060C944A07B2
:100EB0000F931F930091EB011091EC012091ED0134
:100EC0003091EE01602B712B822B932B1F910F9190
:100ED0000C944A070F931F930091EB011091EC01C2
:100EE0002091ED013091EE01602371238223932341
:100EF0001F910F910C944A070F931F930091EB01E0
:100F00001091EC012091ED013091EE0160277127E5
:100F1000822793271F910F910C944A070C94450741
:100F20000E948E076093E7017093E8018093E901C6
:100F30009093EA010C94E60660E070E0CB010C941B
:100F400090070F931F9341E050E060E070E08A014A
:100F50009B0104C0000F111F221F331F8A95D2F777
:100F6000C901B8011F910F910C9490070F931F9323
:100F700041E050E060E070E004C0440F551F661F80
:100F8000771F8A95D2F78091E7019091E801A091AF
:100F9000E901B091EA018A019B01082B192B2A2B48
:100FA0003B2BC901B8011F910F910C9490070F932F
:100FB0001F9341E050E060E070E004C0440F551F13
:100FC000661F771F8A95D2F740955095609570956A
:100FD0008091E7019091E801A091E901B091EA01C7
:100FE0008A019B01082319232A233B23C901B80145
:100FF0001F910F910C9490070F931F9341E050E0C5
:1010000060E070E004C0440F551F661F771F8A958B
:10101000D2F78091E7019091E801A091E901B091A8
:10102000EA018A019B01082719272A273B27C901C2
:10103000B8011F910F910C9490070F931F9300918B
:10104000E7011091E8012091E9013091EA01602B5C
:10105000712B822B932B1F910F910C9490070F9360
:101060001F930091E7011091E8012091E90130916F
:10107000EA0160237123822393231F910F910C9423
:1010800090070F931F930091E7011091E8012091C1
:10109000E9013091EA0160277127822793271F9188
:1010A0000F910C949007089528E0929F800D1124D1
:1010B000E82FE695E695E695877051E001C0550F5B
:1010C0008A95EAF785E0E89FF0011124EE56FE4F7D
:1010D00020E030E070E04081CB01022E02C0969506
:1010E00087950A94E2F78170819584278523842768
:1010F00081932F5F3F4F2530310569F7089528E030
:10110000929F800D1124682F669566956695982F9D
:10111000977085E0689FB001112440E050E080E0C6
:10112000FB01E40FF51FEE56FE4F208130E0092E43
:1011300002C0369527950A94E2F721703327042ED2
:1011400001C0220F0A94EAF7822B4F5F5F4F4530B0
:10115000510531F70895BF92CF92DF92EF92FF923F
:101160000F931F93CF93DF938C01C090E701D09032
:10117000E801E090E901F090EA018091EB019091A3
:10118000EC01A091ED01B091EE01C82AD92AEA2A1A
:10119000FB2ACFE1D0E0D701C6010C2E04C0B695E2
:1011A000A795979587950A94D2F780FD04C021975B
:1011B00090F7B12C07C0BC2EB8018C2F0E94DB0F1A
:1011C0000197A9F38B2DDF91CF911F910F91FF9084
:1011D000EF90DF90CF90BF900895CF93DF93EC0115
:1011E0000E94AB08BE010E94DB0FDF91CF910895F2
:1011F0001F93CF93DF93EB0190919101992321F0FD
:10120000CB010E94ED0813C0882349F0CB010E9456
:10121000AB08182F682FCE010E94540804C0CB01E0
:101220000E947F08182FBE01812F0E94DB0FDF91E3
:10123000CF911F9108951F93CF93DF93C091EF013A
:1012400016E08091F001C81799F0D0E01C9FF001E2
:101250001D9FF00D1124EF50FE4F4081518162819E
:101260007381848195810E9434072196C770E9CFEC
:10127000DF91CF911F910895409121025091220258
:1012800060912302709124028091250290912602A0
:101290000C943407EF92FF920F931F93CF93DF9339
:1012A0008091260282958F7009F065C0809123029B
:1012B000882309F460C08091EF01F090F001109153
:1012C000210200912202609124027091250291E096
:1012D0001F3F09F090E0C0910001D0910101292F3A
:1012E00096E0E92E8F1509F446C06115710521F0CD
:1012F0000F3F21F030E003C031E001C0322F90E019
:1013000030FD36C0E89EF001E99EF00D1124DF01AA
:10131000AF50BE4F11963C911197301329C03C91AC
:10132000311326C012963C911297311121C01396A9
:101330004D915C911497461B570B4C175D07C0F4F9
:10134000809126028F70806180932602EA50FE4FC2
:1013500080818F708061808381E292E00E94B2067A
:10136000DF91CF911F910F91FF90EF900C941B098B
:1013700001968770B7CFDF91CF911F910F91FF90AA
:10138000EF9008959F92AF92BF92CF92DF92EF922B
:10139000FF920F931F93CF93DF93CDB7DEB7619783
:1013A0000FB6F894DEBF0FBECDBF8C0185E0F8010B
:1013B000DE011D9601900D928A95E1F7D8011296F3
:1013C000EC9090912102E091220220912402309130
:1013D00025022115310531F0EF3F31F481E09F3FC7
:1013E00019F403C081E001C080E0B82FB1709B2EDA
:1013F00080FD47C1D8014C9111965C9111971396CD
:10140000AD90BC90149781E2C82E82E0D82EF09067
:101410002302B501621B730B209100013091010181
:10142000FF2009F4D9C0809126026217730708F0E3
:1014300095C0282F207F09F052C05E1313C04913B6
:1014400011C0FE2CE1100EC08F70806180932602C7
:101450000E943C09C6010E94B20680912602F80152
:1014600085834DC1AB2831F05F3F31F481E04F3FC0
:1014700019F403C081E001C080E080FD03C081E079
:101480008E2502C080E090E0F82FF170FF2E80FFE3
:101490001CC08091EF012091F00136E0821709F421
:1014A0000BC190E0389FF001399FF00D1124EF50EF
:1014B000FE4F6181561306C06081461303C06281EE
:1014C000E61203C001968770E9CFFE2CEE2009F4E6
:1014D00016C18091260281608093260254C05E135B
:1014E00006C0491304C0E11002C0F80199C0C80148
:1014F0000E941D07882361F1EE2051F12091260200
:10150000822F82958F7090E0029774F08091210273
:101510009091220298878F831986BB86AA862C8792
:10152000CE0107960E94B20686E0F801A1E2B2E081
:1015300001900D928A95E1F70E944A090E943C09A8
:101540000AC05E1711F1C8010E941D0781112CC04D
:10155000C8010E94B206FF24F394D1C0282F207F37
:1015600081F77A2DB98AA88A6E2D89890E9425076C
:1015700081E292E00E94B20686E0D6011D928A9531
:10158000E9F70E943C09F12CBAC04913DCCFE11005
:10159000DACFF8018583C8010E94B20686E0D60141
:1015A0001D928A95E9F7ABC0EE2091F220912602B8
:1015B000822F82958F7090E002970CF4B5CF8091C6
:1015C0002102909122029A8389831B82BD82AC8280
:1015D0002E83CE010196A6CF6217730708F044C090
:1015E000FE2CEE2009F4B4CF5E1330C049132EC098
:1015F0002091260220FD21C0822F82958F70482FD6
:1016000050E041155105C9F0F80125834F305105CF
:1016100041F08F5F982F9295907F822F8F70892B4A
:101620008583C8010E94B20686E0F801A1E2B2E01B
:1016300001900D928A95E1F73CC086E0F801A1E2A5
:10164000B2E001900D928A95E1F759C0C8010E945D
:101650001D07811169CF8091260281608093260247
:10166000C8010E94B2064BC07A2DB98AA88A6E2D95
:1016700089890E94250786E0D6011D928A95E9F79F
:1016800018C0EE2009F464CFC8010E941D07F82E8F
:10169000882309F45DCF86E0F801A1E2B2E0019071
:1016A0000D928A95E1F781E292E00E94AB030E94DD
:1016B0004A090E943C0923C04D875E878D859E851F
:1016C0000E94ED08292F22952F70223028F49F7058
:1016D00039F0811105C00BC0243028F49F7049F403
:1016E000805E883020F0C8010E94B2069F2CF92C41
:1016F00006C0D80115969C91907F91F7F8CF8F2D59
:1017000061960FB6F894DEBF0FBECDBFDF91CF91CB
:101710001F910F91FF90EF90DF90CF90BF90AF900F
:101720009F9008951F93CF93DF93CDB7DEB72C978B
:101730000FB6F894DEBF0FBECDBF4F8358876987C1
:101740007A878B879C87CE0107960E94C2098823DF
:10175000D1F09F8188852A853B85232B31F08F3FEF
:1017600031F481E09F3F19F403C081E001C080E0C3
:1017700080FD47C04F81588569857A858B859C851A
:101780000E9434073EC086E0FE013796DE011196C6
:1017900001900D928A95E1F7FF81E8856A857B8546
:1017A0006115710531F0EF3F31F481E0FF3F19F42D
:1017B00003C081E001C080E080FD23C02091F001E2
:1017C00030E0C9010196877099274091EF0150E000
:1017D00084179507F1F1F983EA837D836C8396E0A2
:1017E000929FD001939FB00D1124AF50BE4FFE01C8
:1017F000319601900D929A95E1F78093F0010E9445
:101800001B0916E08091EF019091F001891771F1A9
:10181000189FC00111248F509E4F0E94C209882337
:1018200029F1E091EF011E9FF0011124EF50FE4FCE
:101830004081518162817381848195810E94340746
:101840008091EF0190E00196877099278093EF01D6
:10185000D9CF0E94FE061092F0011092EF01E1E252
:10186000F2E086E0DF011D928A95E9F72C960FB62B
:10187000F894DEBF0FBECDBFDF91CF911F910895C9
:1018800080914702859585958595089580914702B9
:101890008770089590914702977081E009F480E085
:1018A000089580916A02089590916A02892B80932D
:1018B0006A020895809590916A02892380936A0252
:1018C000089510926A02089590916902892B80937D
:1018D0006902089580959091690289238093690235
:1018E000089510926902089580914802089508951C
:1018F0000C94770C0C94780C9091E70292FD08C040
:1019000090914802981721F0809348020C947A0C29
:10191000089580914802882329F01092480280E0BF
:101920000C947A0C0895CF93DF93E0910201F0912B
:10193000030180916A028083E0910201F09103012A
:10194000908180916902892B80838091480288234D
:1019500081F0E0910201F09103019081892B808355
:1019600080910201909103010E94D51781110E947C
:10197000890CC0910201D091030140E250E067E27E
:1019800072E0CE010E94AE20892B69F080E2FE0158
:10199000A7E2B2E001900D928A95E1F7CE01DF91C6
:1019A000CF910C948117DF91CF9108950C94770C0F
:1019B0009091E70292FD10C098E0899F9001112458
:1019C000262B209347020E94B607809147028595F7
:1019D000859585950C94D60C0C94B6071092470209
:1019E00080E00C94D60C209147028095822380934E
:1019F0004702982F977099F430E0482F082E000C7A
:101A0000550B2417350759F09091E70292FD07C056
:101A10008595859585950E94D7070C94EE0C0895C1
:101A20009091E70292FB222720F9281769F080FBAA
:101A300092F99093E7028091E6029091E7020E946A
:101A4000580D82E00C94F30C08958091E70282FB1C
:101A5000882780F991E089270C94100D81E00C947F
:101A6000100D80E00C94100D80E090E00E94C320E7
:101A700021E0893E9E4F09F020E0822F089582E008
:101A800090E00C94BB2083E090E00C94BB20CF93BB
:101A900084E090E00E94BB20C82F82E290E00E9488
:101AA000BB202C2F30E0A901582BCA01CF910895FB
:101AB000CF93C92F682F84E090E00E94C9206C2F3B
:101AC00082E290E0CF910C94C920AB01BC018FE081
:101AD00090E00C94DB20AB01BC0183E190E00C941E
:101AE000DB2060E070E0CB010C946B0D60E070E0F7
:101AF000CB010E94650D0C94710D69EE7EEF80E0C4
:101B000090E00E94E72060E082E090E00E94C9201F
:101B100060E083E090E00E94C9201092EB011092F7
:101B2000EC011092ED011092EE0160E084E090E093
:101B30000E94C92060E082E290E00E94C92060E03B
:101B400085E090E00E94C92060E086E090E00E947D
:101B5000C9206FEF87E090E00E94C92040E050E08C
:101B6000BA0188E090E00E94DB2060E08DE090E028
:101B70000E94C92040E050E0BA0188E190E00E9454
:101B8000DB2060E087E190E00E94C92040E050E067
:101B9000BA018CE190E00E94DB2060E070E080E21E
:101BA00090E00E94E72040E050E0BA0188E190E038
:101BB0000E94DB200C94760D0C947D0D682F8EE036
:101BC00090E00C94C9200E943A19609380027093AF
:101BD0008102809382029093830260937C027093CF
:101BE0007D0280937E0290937F02089585B780687E
:101BF00085BF85B7806885BF089581E008950C94FE
:101C0000FD0D08950C94010E0C94010E0C94040E1D
:101C10000C94010E0C94080E0C94010E0E94F60D0B
:101C200087EB90E10E946B170E940C0E0C940A0E39
:101C30000E94020E0C94010E0E94BA100C944E03E6
:101C40000E9425190E94F6010E941C0E0C94060E9B
:101C50008F929F92AF92BF92CF92DF92EF92FF92BC
:101C60000F931F93CF93DF93CDB7DEB72A970FB6AD
:101C7000F894DEBF0FBECDBF0E940602982E8111E0
:101C80000E94E30D8BE6A82E82E0B82E00E010E063
:101C9000802E802F0E948102D82EF501C1905F0115
:101CA000C826B1F40F5F1F4F0131110589F78FEF7F
:101CB00089838A831B820E942E198160782F9D83DD
:101CC0008C8349815A816B818D810E9461032FC071
:101CD0008091840281FD0E948702E12CFF24F3940D
:101CE0008C2D8F21F1F00E94FF0D882399F0EE8258
:101CF0008F82DF2081E009F480E088870E942E191E
:101D00008160782F9A8789874E815F8168858A856F
:101D10000E946103F801E559FD4F8081F826F082A9
:101D200006C0E394FF0CF8E0EF12DACFBBCF81E0FE
:101D3000911001C080E02A960FB6F894DEBF0FBE66
:101D4000CDBFDF91CF911F910F91FF90EF90DF906A
:101D5000CF90BF90AF909F908F9008950E94280ED3
:101D60000E945F120C945603CF93DF930E94E00F02
:101D7000EC01811521E5920708F045C0811530E599
:101D8000930708F094C0883E910528F5803E9105A0
:101D900008F0F8C0883A910570F4853A910508F08A
:101DA0007CC08130910509F475C008F4E8C004973F
:101DB00008F0E8C0E4C08F3B910508F0E0C0C85AC5
:101DC000D0E0CC0FDD1FC65BDE4F0990D881C02D5F
:101DD000CE019464D8C0811540E2940758F481156F
:101DE00051E0950708F0CEC08D3E910508F4C7C0BC
:101DF0009065C9C0C11580E4D80708F4C0C0DF7081
:101E0000CE01906AC0C0811525E59207A8F481151E
:101E100034E5930708F095C0811543E5940708F071
:101E20007BC0811552E5950708F061C0D82FCC27FB
:101E3000CE01816F906AA7C0C11589E5D807A0F4CB
:101E4000C11528E5D20708F082C0C11536E5D307D1
:101E500008F095C08C2F0E9474108F7190E0D82FDD
:101E6000CC27CE0190628FC0C1154AE5D40708F493
:101E700074C0CE0190568115904208F080C08D2F1D
:101E80008F710E947410DD27D0628F71AE01582BC4
:101E9000CA0179C081E090E076C0C55AD0E0C85848
:101EA000DE4F8881C82FD0E0CE0190646CC074E012
:101EB000969587957A95E1F7282F23703C2F3370FC
:101EC00081E090E002C0880F991F3A95E2F79C6884
:101ED000AC01522B9A019C2F9F709695969550E2DB
:101EE000959FE0011124C9018C2B9D2B4CC0837060
:101EF000992721E030E002C0220F331F8A95E2F7D4
:101F00009C2F9695969580E2989FE0011124C22B14
:101F1000D32BCE019C6837C08370992721E030E035
:101F200002C0220F331F8A95E2F79C2F9695969553
:101F300040E2949FE0011124C22BD32BCE019A687A
:101F400022C0D82FCC27CE01846F906A1CC0DC2F12
:101F5000CC27CE01806F906A16C08C2F8F700E94A4
:101F6000741094E0D695C7959A95E1F7CF70D0E0BC
:101F7000DC2FCC27D0699E01282BC90104C080E04A
:101F800090E001C0CE01DF91CF910895E72FF0E0FE
:101F900091E1899FE00DF11D112483E0EE0FFF1FF9
:101FA0008A95E1F7E60FF11DEE0FFF1FEA51FF4F93
:101FB0008591949108950E94C60F0E94B40E0895D1
:101FC0008238910569F1B0F48133910509F46DC04F
:101FD00048F48932910509F463C08A32910509F405
:101FE00069C008958533910509F455C08933910579
:101FF000B9F00895833E910569F138F4803E91056A
:10200000B1F0823E910509F10895863E9105A9F14E
:10201000873E9105B9F1843E910509F064C023C063
:102020002091E60220FD4FC021FD4DC00895809112
:10203000E60280FD44C08091E70280FF44C08091A9
:10204000E60284FD42C083EE4DC08091E60282FF2D
:1020500038C0F5CF8091E60282FD33C08091E7025F
:1020600080FD31C0ECCF8091E70281FF32C08091CA
:10207000E60284FD2AC087EE35C08091E60283FF28
:1020800026C0F5CF8091E60283FD21C08091E70252
:1020900081FD1FC0ECCF8091E60285FD1CC01DC0F4
:1020A0008091E60285FD19C016C08091E60286FD8A
:1020B00016C017C08091E60286FD13C010C089E3E8
:1020C00011C082EE0FC080EE0DC080E00BC086EE26
:1020D00009C084EE07C089E205C085E303C08AE237
:1020E00001C081E390E008959091E60292FF0DC057
:1020F000282F2871283019F4877F846006C0282F84
:102100002471243011F48B7F886093FF0DC0282F39
:102110002871283119F4877E846106C0282F247124
:10212000243111F48B7E88612091E70220FF0DC0DD
:10213000382F3871383019F4877F816006C0382F06
:102140003171313011F48E7F886021FF0DC0282F4E
:102150002871283119F4877E816106C0282F2171EA
:10216000213111F48E7E886194FD877E089580E090
:10217000089508950E94340D811102C00E94DC0D63
:102180000E943F0D809384020E94470D9093E702C6
:102190008093E6020E94B9100E94430D682F70E000
:1021A00080E090E00E9456076091E7017091E8019D
:1021B0008091E9019091EA010C948E070E94461BE0
:1021C0000E94200E0C94521B0E94561B0E94AE0EC1
:1021D0000C94701B0E94CC180E942D1B0E940E0EA6
:1021E0000E94DE100E94E4100E94180EFBCF809126
:1021F0008B0280FF06C06091090170E0660F771FB7
:1022000026C081FF04C06091090184E005C082FFFF
:1022100007C06091090188E0689FB001112417C0D0
:1022200090918A029923D1F060910801961788F75E
:102230002091090188E0289F90011124929FA0011C
:10224000939F500D112470E0CA010E9480206038D5
:10225000710540F46115710519F406C068E070E07D
:10226000862F08958FE7089581E0089580918B026D
:1022700080FF08C06091050170E0759567957595C0
:10228000679521C081FF06C06091050170E07595DA
:10229000679519C082FF04C06091050170E010C00D
:1022A00090918902992399F0609104019617A0F703
:1022B00080910501899FC001112470E00E94802057
:1022C0006038710540F46115710519F406C061E0CC
:1022D00070E0862F08958FE7089581E008958D3E80
:1022E00021F40E94F710819504C08E3E29F40E94CB
:1022F000F71080938F0208958F3E21F40E94F7100B
:10230000819504C0803F29F40E94F71080938E02CB
:102310000895893F19F40E94361105C08A3F31F4AF
:102320000E94361181958093900208958B3F21F48D
:102330000E943611819504C08C3F29F40E94361109
:102340008093910208959FE0980F983078F421E0EF
:1023500030E0A90102C0440F551F9A95E2F7CA0167
:1023600090918D02892B80938D0208958D3F21F4E9
:1023700080918B0281600BC08E3F21F480918B0293
:10238000826005C08F3F29F480918B028460809326
:102390008B0208958D3E39F490918F0297FF35C0DE
:1023A00010928F0259C08E3E29F490918F02191617
:1023B000BCF32BC090918E028F3E29F497FF25C06D
:1023C00010928E0249C0803F19F41916CCF31DC03B
:1023D00090919002893F29F41916BCF41092900252
:1023E0003BC08A3F19F497FF10C0F8CF8B3F39F4F8
:1023F0009091910297FF09C0109291022DC08C3FDD
:1024000021F4909191021916BCF39FE0980F983037
:1024100080F421E030E0A90102C0440F551F9A95D5
:10242000E2F7CA01809590918D02892380938D02F5
:1024300013C08D3F21F480918B028E7F0BC08E3FA5
:1024400021F480918B028D7F05C08F3F29F480910C
:102450008B028B7F80938B0280918E02811106C04C
:1024600080918F02811102C010928A0280919002A5
:10247000811106C080919102811102C010928902DF
:1024800008950E942E1920918E02211104C02091DE
:102490008F02222321F0909388028093870220915B
:1024A0009002211104C020919102222321F09093E7
:1024B0008602809385028CE892E00C949B17EF9241
:1024C000FF920F931F93CF93DF9300D000D000D0E3
:1024D000CDB7DEB786E0ECE8F2E0DE0111960190C0
:1024E0000D928A95E1F7E0908E02F0908F020091B4
:1024F00090021091910210928E0210928F0210920F
:10250000900210929102E11003C0FF2009F45DC017
:1025100080918702909188020E944619AC019091A7
:102520008A02992339F020910A0130E024173507F7
:1025300058F04BC020910B018AE0289F9001112494
:102540002417350718F041C09F3F19F09F5F909303
:102550008A02EE2061F00E94F7101E1414F09FEF23
:1025600001C091E0989F902D112490938E02FF203E
:1025700061F00E94F7101F1414F09FEF01C091E06A
:10258000989F902D112490938F0230918E023323C7
:10259000E1F020918F022223C1F045EB3403C0010A
:1025A0001124992319F090938E0203C081E0809347
:1025B0008E0235EB2303C0011124992319F0909367
:1025C0008F0203C081E080938F02011103C01123A9
:1025D00009F45DC080918502909186020E9446199F
:1025E000AC0190918902992339F02091060130E0E5
:1025F0002417350758F04BC0209107018AE0289F27
:10260000900111242417350718F041C09F3F19F09D
:102610009F5F90938902002361F00E94361110168B
:1026200014F09FEF01C091E0989F902D112490939A
:102630009002112361F00E943611111614F09FEFE1
:1026400001C091E0989F902D1124909391023091B8
:1026500090023323E1F0209191022223C1F045EB57
:102660003403C0011124992319F09093900203C000
:1026700081E08093900235EB2303C001112499235C
:1026800019F09093910203C081E0809391028091B0
:102690008E0281110BC080918F02811107C0809141
:1026A0009002811103C08091910281110E94411218
:1026B000EB82FC820D831E8386E0FE013196ACE83E
:1026C000B2E001900D928A95E1F726960FB6F89444
:1026D000DEBF0FBECDBFDF91CF911F910F91FF9055
:1026E000EF900895ECE8F2E086E0DF011D928A9514
:1026F000E9F710928A021092890210928B020895D3
:10270000CF93DF93EC01FB018281882309F43CC164
:10271000C430FDE5DF0760F4CB3F9CE5D90788F4C2
:102720009E0122503C452431310508F02EC109C0DC
:10273000C236EDE5DE0729F0C63AFDE5DF0709F010
:1027400024C10E94470D9093E7028093E602C131B5
:102750008CE5D80709F4C6C008F042C0C930ECE5E2
:10276000DE0709F49BC000F5C5308CE5D80709F4F5
:1027700085C078F4C330ECE5DE0709F478C008F0D2
:102780007AC0C230DC4509F0F5C08091E602816074
:10279000EFC0C7309CE5D90709F478C008F07AC0CB
:1027A0008091E6028061E4C0CD30FCE5DF0709F4EA
:1027B00087C058F4CB309CE5D90709F479C008F0FC
:1027C0007BC08091E60288606FC0CF30FCE5DF07F8
:1027D00009F480C008F082C08091E602877FC8C0FB
:1027E000CE3F9CE5D90709F471C000F5C531FCE581
:1027F000DF0709F485C068F4C3319CE5D90709F403
:1028000075C008F095C00E94FE068091E6028F77A1
:10281000AFC0CC3FFCE5DF07A9F108F054C0CB3FC7
:10282000DC4509F0A7C08091E70240C0C230EDE569
:10283000DE0709F489C058F4C1158DE5D80709F4FD
:102840005AC008F069C08091E70282602FC0C2368A
:10285000EDE5DE0709F47CC0C63AFDE5DF0709F4C3
:1028600081C0C330DD4509F085C080E06EC0809135
:10287000E60282607DC08091E60216C08091E60289
:10288000886076C08091E70282604FC08091E60246
:1028900080626EC08091E60280646AC00E94FE067B
:1028A0008091E602806864C0846062C081603DC03F
:1028B0008091E6028E7F5CC08091E6028D7F58C0D9
:1028C0008091E60216C08091E70218C08091E7026D
:1028D0008D7F2BC08091E6028F7E4AC08091E602F8
:1028E0008F7D46C08091E6028F7B42C08091E602D8
:1028F000877F8B7F3DC08091E7028D7F8E7F15C0E3
:102900008091E60282FB222720F991E0922790FB3A
:1029100082F990FB83F92CC08091E702982F909563
:1029200091708E7F892B90FB81F98093E70222C002
:102930000E94FE068091E60287FB222720F991E0A3
:10294000922790FB87F914C081E00E94DE0D12C02F
:102950008091E60284FB222720F991E0922790FBE8
:1029600084F906C08091E602982F909590FB80F93B
:102970008093E6028091E6029091E7020E94580D52
:102980000E94FE0680E001C081E0DF91CF910895B2
:102990009FB7F8942091920280919302821761F080
:1029A00030E0F901EC56FD4F80812F5F3F4F2F71D2
:1029B00033272093920201C080E09FBF0895CF93F8
:1029C000DF93EC010E945916882341F0209731F0E3
:1029D00085E08A95F1F700002197F4CFCE01DF91D1
:1029E000CF910895CF93DF93C2E3D0E00E945916B0
:1029F000811108C0209731F085E08A95F1F7000039
:102A00002197F4CFCE01DF91CF9108950E94561601
:102A10000E9467165D985A9886E78093CA001092C4
:102A2000C8001092CD001092CC0080E98093C900BC
:102A300008958AE1815011F40C94C8143FB7F894BA
:102A400020919302909192023FBF2913F5CFEFE9B5
:102A5000FFE03197F1F700C00000ECCFEF92FF925A
:102A60000F931F93CF93DF93E82E1092B40210922E
:102A7000CA008091C900877E8093C9000E945316C6
:102A80000E9467168FE891E00197F1F700C00000FF
:102A90000E9464160E94561680E197E20E94DF149D
:102AA000892B11F48AE077C0C0E0D0E011E0F12C6E
:102AB00001E090E59A95F1F7C7010C2E02C09595BB
:102AC00087950A94E2F780FF04C010270E946716DA
:102AD00002C00E9464160E94F214892B11F482E055
:102AE0005AC082E390E00E94DF14892B11F483E046
:102AF00052C02196C830D105E1F680E58A95F1F7FC
:102B0000112319F00E94671602C00E9464160E94E9
:102B1000F214892B11F484E03EC082E390E00E941D
:102B2000DF14892B11F485E036C090E59A95F1F712
:102B30000E946716C2E3D0E00E946A16882341F023
:102B4000209741F025E02A95F1F700002197F4CF76
:102B5000CD2B11F486E01FC082E390E00E94DF14C9
:102B6000892B11F487E017C00E94F214892B19F009
:102B7000C2E3D0E009C088E00EC0209759F085E09C
:102B80008A95F1F7000021970E946A168823A9F31D
:102B9000CD2BE9F489E08093B4020E9456160E947E
:102BA00067165D985A9886E78093CA001092C8000D
:102BB0001092CD001092CC0080E98093C90080E093
:102BC000DF91CF911F910F91FF90EF9008950E9498
:102BD00056160E9467165D985A9886E78093CA0039
:102BE0001092C8001092CD001092CC0080E9809322
:102BF000C900DF91CF911F910F91FF90EF900C943E
:102C000019152FB7F89490919302809192022FBFDB
:102C1000981721F01092B4020C94C81480E28093AB
:102C2000B40280E008951F920F920FB60F92112404
:102C30002F933F934F935F936F938F939F93EF9354
:102C4000FF938091C8005091CE008C71A9F44FB7CA
:102C5000F8948091930290E09C012F5F3F4F2F7179
:102C6000332760919202621731F0FC01EC56FD4F60
:102C70005083209393024FBFFF91EF919F918F91CB
:102C80006F915F914F913F912F910F900FBE0F90D9
:102C90001F901895CF93C82F8DEE0E942E158C2F64
:102CA000CF910C942E155D98559A089555985D9A7C
:102CB000089555985D9A85E08A95F1F7000089B1ED
:102CC00085FB882780F908955A98529A089552985A
:102CD0005A9A089552985A9A85E08A95F1F7000019
:102CE00089B182FB882780F90895CF93DF938631DD
:102CF0009C4541F5EB010E94510C982F8A8120914F
:102D0000020130910301882379F09A7A81E009F475
:102D100080E08093B502911102C069E201C065E3D1
:102D2000C9010E946B180AC08091B502811102C0CE
:102D300069E201C065E3C9010E9476180E94930C04
:102D400080E001C081E0DF91CF9108950F931F9340
:102D5000CF93DF93C42FD22FFC0182818823C9F047
:102D60004093B8020E942E199093B7028093B60246
:102D700080E28C0F883008F057C0C77081E001C036
:102D8000880FCA95EAF7DF91CF911F910F910C94AC
:102D90005B048091B802481330C08091B6029091D4
:102DA000B7020E944619883C910538F510E21D0FC4
:102DB000CD17B9F080E28C0F883040F4C77081E005
:102DC00001C0880FCA95EAF70E946204183028F5FE
:102DD00081E09D2F977001C0880F9A95EAF70E94B5
:102DE0005B04802F0E9452041830F0F4D77081E009
:102DF00001C0880FDA95EAF70AC080E28C0F8830AC
:102E000098F4C77081E001C0880FCA95EAF7DF9196
:102E1000CF911F910F910C946204802FDF91CF917D
:102E20001F910F910C945204DF91CF911F910F913C
:102E300008950F939C01CB01243F4CE5340731F1F9
:102E400088F4293DFCE53F07D9F02A3D4CE53407DD
:102E500079F1283D3C45A9F506E221EE41EE68ED09
:102E60007CE52BC0263FFCE53F07E1F0A8F0273FBB
:102E70003C4539F507E225EE46EE67EF7CE51DC0DF
:102E800007E225EE45EE69ED7CE517C006E221EE8E
:102E900040EE64EF7CE511C007E225EE44EE65EFFD
:102EA0007CE50BC006E221EE42EE66EF7CE505C054
:102EB00008E221E045EE6AED7CE50E94A61680E07E
:102EC00008C0FC018281882319F01092B80201C069
:102ED00081E00F91089590937D0180937C01089586
:102EE0009093BE028093BD020895E091BD02F091DF
:102EF000BE02309721F00190F081E02D099480E02E
:102F00000895E091BD02F091BE02309799F02091B2
:102F10001801222359F02091E60227FF07C0DC01A7
:102F20002C9111962C93119726E02C930280F3811B
:102F3000E02D09940895E091BD02F091BE02309712
:102F400039F022E0DC012C930480F581E02D099416
:102F500008952091BB023091BC022817390771F007
:102F60009093BC028093BB02E091BD02F091BE023F
:102F7000309721F00680F781E02D09940895209183
:102F8000B9023091BA022817390771F09093BA024A
:102F90008093B902E091BD02F091BE02309721F01A
:102FA0000084F185E02D09940895FC01329680910A
:102FB0001801882331F08091E60287FF02C09EE16C
:102FC00001C096E080E0915028F021912223D9F3AE
:102FD0008F5FF9CF0895662351F1209118012223C4
:102FE000E9F02091E60227FF19C0462F4695469545
:102FF00046954E31E0F4677021E030E002C0220FC8
:10300000331F6A95E2F7FC01E40FF11D828190E025
:103010002823392381E0232B69F409C0FC0132966F
:1030200008962191621729F0E817F907D1F780E097
:10303000089581E008959C01FC0132969FEF80E0A5
:103040004191461789F09F3F19F4411101C0982F13
:103050008F5F8630A9F79F3F39F0F901E90FF11D25
:1030600097FDFA956283089508959C012A5F3F4F6A
:10307000FC014281461301C0128201968217930718
:10308000B9F70895262F2695269526952E3168F4B2
:10309000FC01E20FF11D677021E030E001C0220F5A
:1030A0006A95EAF78281282B22830895262F269598
:1030B000269526952E3170F4FC01E20FF11D677004
:1030C00021E030E001C0220F6A95EAF72095828165
:1030D00028232283089520911801222329F020918A
:1030E000E60227FD0C9442180C941B18209118013D
:1030F000222329F02091E60227FD0C9456180C9407
:10310000351820911801FC013296222331F080916C
:10311000E60287FF02C08EE101C086E0DF011D925A
:103120008A95E9F7089508950C94931883E08093A5
:10313000BF020C949418811102C081E001C082E0AA
:103140008093BF020C9494180C949B1881E0809398
:10315000BF020C9494180C94A61808950C94AD1802
:103160000C94AE180C94AD180C94AD180C94AD18CA
:10317000CF930E94B4180E9406020E94B218C0E0C9
:103180008C2F0E948102811104C0CF5FC131C1F731
:1031900001C081E0CF91089508951F920F920FB65C
:1031A0000F9211248F939F93AF93BF938091C0028E
:1031B000811113C08091E8029091E902A091EA0286
:1031C000B091EB024196A11DB11D8093E80290934E
:1031D000E902A093EA02B093EB02BF91AF919F91F5
:1031E0008F910F900FBE0F901F9018958091F00255
:1031F000843031F10E9446031092C00220E488E13D
:1032000090E00FB6F894A895809360000FBE2093CD
:10321000600083B7817F846083BF83B7816083BF91
:103220007894889583B78E7F83BF0FB6F894A8955E
:1032300080916000886180936000109260000FBEF2
:1032400008950E94FE060C944A0382E084BD93E038
:1032500095BD9AEF97BD80936E0008952FB7F894AF
:103260008091E8029091E902A091EA02B091EB020C
:103270002FBF08952FB7F8946091E8027091E9028A
:103280008091EA029091EB022FBF08959C014FB705
:10329000F8948091E8029091E902A091EA02B0913D
:1032A000EB024FBF821B930B089578941F920F92ED
:1032B0000FB60F9211248F939F93AF93BF9380917A
:1032C000E8029091E902A091EA02B091EB02019626
:1032D000A11DB11D8093E8029093E902A093EA0238
:1032E000B093EB02BF91AF919F918F910F900FBE62
:1032F0000F901F90189581E08093E00080E280930A
:10330000D8001092C9008FE19EE40197F1F700C048
:10331000000087E090EBDC018093F9029093FA02C1
:10332000A093FB02B093FC029CE088E10FB6F894F6
:10333000A895809360000FBE90936000FFCF8091AE
:10334000E4020895089522E02093E9002FEF3091E0
:10335000E800215035FD06C035ED3A95F1F7000043
:103360002111F5CF2091E80025FF0BC040E050E08F
:1033700066E070E00E94E21B8091E8008E77809307
:10338000E8000895CF93DF9320911801222339F0AC
:103390002091E60227FF03C060E222E002C068E05D
:1033A00021E02093E9002FEF3091E800215035FD16
:1033B00006C035ED3A95F1F700002111F5CF2091C7
:1033C000E80025FF1DC0EC0180911801811105C0A6
:1033D00040E050E068E070E003C070E040E050E0A2
:1033E000CE010E94E21B8091E8008E778093E80076
:1033F00080E2FE01A4ECB2E001900D928A95E1F723
:10340000DF91CF9108958093C1027093C3026093BE
:10341000C2028091F002843001F582E08093E900DD
:103420008FEF9091E800815095FD06C095ED9A953B
:10343000F1F700008111F5CF8091E80085FF0DC004
:1034400040E050E063E070E081EC92E00E94E21B1B
:103450008091E8008E778093E8000895BC0184E0B5
:103460000C94031ABC0183E00C94031A8091EF02C0
:10347000811109C00E94731D0E94D01D8091E2003D
:1034800084608093E20008951092EF0208950C94F6
:10349000AB186091EC0281E0611101C080E00C94F6
:1034A00096189091F00281E0943009F080E06091EC
:1034B000EC020C949B1842E061EC81E00E94EC1C51
:1034C00042E261EC82E00E94EC1C9091F00281E00B
:1034D000943009F080E06091EC020C94A418809183
:1034E000F202833009F461C030F4813071F082302F
:1034F00009F49AC008958A3009F486C08B3009F423
:103500006CC0893009F0A8C020C08091F102813AD6
:1035100009F0A2C08091E800877F8093E800809145
:10352000F5029091F602892B21F460E284EC92E09E
:1035300003C060E080E090E070E00E942D1C80916C
:10354000E8008B778093E80008958091F102813242
:1035500009F082C08091F5029091F602029708F07E
:103560007BC08091E800877F8093E8008091E8002D
:1035700082FD05C08091F0028111F8CF6DC02091CD
:10358000F3008091F20090E0922B029731F4809149
:10359000F100813011F0863021F48091F1008093A8
:1035A000E4028091E8008B7753C08091F102813A68
:1035B00009F052C08091F5029091F602892B09F032
:1035C0004BC08091E800877F8093E8008091E800FD
:1035D00080FFFCCF8091180136C08091F1028132CA
:1035E000D9F58091F5029091F602892BA9F5809189
:1035F000E800877F8093E8000E94211D8091F302FC
:10360000809318010C94FE068091F102813221F51D
:103610008091E800877F8093E8000E94211D8091BF
:10362000F4028093E50208958091F102813AA1F4B9
:103630008091E800877F8093E8008091E80080FF18
:10364000FCCF8091E5028093F1008091E8008E77B5
:103650008093E8000C94211D089584B7877F84BF70
:103660000FB6F894A89580916000886180936000FF
:10367000109260000FBE90E080E80FB6F89480933F
:103680006100909361000FBE0C94A6180E94731DF8
:103690000E94D01DE2EEF0E0808184608083789407
:1036A0000C9465208CE091E00C9470178091F002EE
:1036B0008530A9F48091F002853079F40E94F618E3
:1036C0008091EE028823B1F30E94B818882391F309
:1036D0000E94CC1B0E94FE06EDCF0C942119089588
:1036E00008950C94731B292F332723303105C9F01B
:1036F00060F42130310581F02230310509F044C0F9
:103700008BE390E022E332E043C021323105E1F067
:103710002232310549F138C082E190E02DE632E0F5
:1037200037C099278130910549F028F0029761F55B
:10373000E6EFF1E005C0EEE2F2E002C0E4E2F2E022
:10374000849190E09F0124C06115710541F06130C2
:103750007105D1F489E090E02DE532E019C089E0EF
:1037600090E024E432E014C06115710541F061304D
:10377000710551F486EB90E02FE732E009C080E458
:1037800090E025E333E004C080E090E020E030E00A
:10379000FA0131832083089580E189BD82E189BDEA
:1037A00009B400FEFDCF8091D8008F7D8093D800B2
:1037B0008091E00082608093E0008091E00081FDD4
:1037C000FCCF0895CF92DF92EF92FF920F931F9359
:1037D000CF93DF93EC018B017A010E94401D811190
:1037E00033C0E114F10439F0F70180819181081BA5
:1037F000190BC80FD91FC12CD12C0115110519F1B6
:103800008091E80085FD16C08091E8008E77809356
:10381000E800E114F10449F0F70180819181C80EBC
:10382000D91ED182C08285E00FC00E94401D88232E
:1038300021F30AC089918093F10001501109FFEF33
:10384000CF1ADF0ADACF80E0DF91CF911F910F917D
:10385000FF90EF90DF90CF9008952091F702309184
:10386000F8022617370748F06115710539F42091E1
:10387000E8002E772093E80001C0B901FC0120E0A8
:103880006115710579F18091F0028823F1F185309D
:10389000F1F18091E80083FD3CC08091E80082FD59
:1038A0002EC08091E80080FFEBCF2091F300809143
:1038B000F20090E0922B6115710551F0883091056E
:1038C00038F421912093F100615071090196F3CFF2
:1038D00021E0089709F020E08091E8008E7780933E
:1038E000E800CECF2111CFCF0AC08091F00288230B
:1038F00061F0853061F08091E80083FD0AC080911D
:10390000E80082FFF2CF80E0089582E0089583E02E
:10391000089581E008952091F7023091F80226176A
:10392000370748F06115710539F42091E8002E77CA
:103930002093E80001C0B901FC0120E06115710588
:1039400091F18091F002882309F440C0853009F498
:103950003FC08091E80083FD3DC08091E80082FD7A
:103960002FC08091E80080FFE9CF2091F300809183
:10397000F20090E0922B6115710559F088309105A5
:1039800040F424912093F100319661507109019621
:10399000F2CF21E0089709F020E08091E8008E77CF
:1039A0008093E800CBCF2111CCCF0AC08091F002E8
:1039B000882361F0853061F08091E80083FD0AC0C2
:1039C0008091E80082FFF2CF80E0089582E00895C0
:1039D00083E0089581E00895982F973068F59093DB
:1039E000E900981739F07091EC002091ED005091AA
:1039F000F00003C0242F762F50E021FD02C09F5F0E
:103A0000ECCF3091EB003E7F3093EB003091ED0036
:103A10003D7F3093ED003091EB0031603093EB004F
:103A20007093EC002093ED005093F0002091EE0095
:103A300027FDE5CF80E008958F708093E90081E055
:103A400008958091F10287FF11C08091E80082FD06
:103A500005C08091F0028111F8CF11C08091E8007B
:103A60008B770BC08091F002882349F08091E800A9
:103A700080FFF8CF8091E8008E778093E80008956A
:103A80002091E4003091E50095E64091EC00842F10
:103A9000817040FF23C08091E80080FD1DC08091AF
:103AA000F002882399F0853099F08091EB0085FD34
:103AB00011C04091E4005091E5002417350729F327
:103AC000915011F09A01E1CF84E0089582E00895C9
:103AD00083E0089581E0089580E008954091E80032
:103AE00042FFDDCF08950E94E11D0E94E91DE0EE36
:103AF000F0E0808181608083E8EDF0E080818F7765
:103B0000808319BCA7EDB0E08C918E7F8C9380816F
:103B10008F7E80831092EF0208950F931F93CF93AF
:103B2000DF930E94E11D0E94E91DC8EDD0E088816D
:103B30008F77888388818068888388818F7D888358
:103B400019BC1092F0021092EC021092EE02109248
:103B5000ED0200EE10E0F80180818B7F8083888188
:103B60008160888342E060E080E00E94EC1CE1EE2E
:103B7000F0E080818E7F8083E2EEF0E080818160E2
:103B80008083808188608083F80180818E7F80833C
:103B9000888180618883DF91CF911F910F91089573
:103BA000E8EDF0E080818F7E8083E7EDF0E08081BA
:103BB0008160808384E082BF81E08093EF020C9477
:103BC0008D1DE8EDF0E080818E7F80831092E20011
:103BD00008951092DA001092E10008951F920F925A
:103BE0000FB60F9211242F933F934F935F936F93D0
:103BF0007F938F939F93AF93BF93EF93FF938091A6
:103C0000E10082FF0BC08091E20082FF07C080913B
:103C1000E1008B7F8093E1000E9464208091DA00B4
:103C200080FF1FC08091D80080FF1BC08091DA0008
:103C30008E7F8093DA008091D90080FF0DC080E1F3
:103C400089BD82E189BD09B400FEFDCF81E080938A
:103C5000F0020E94361A05C019BC1092F0020E94B0
:103C6000441A8091E10080FF19C08091E20080FF3A
:103C700015C08091E2008E7F8093E2008091E20087
:103C800080618093E2008091D80080628093D800A8
:103C900019BC85E08093F0020E94491A8091E100EE
:103CA00084FF30C08091E20084FF2CC080E189BD98
:103CB00082E189BD09B400FEFDCF8091D8008F7DDF
:103CC0008093D8008091E1008F7E8093E100809105
:103CD000E2008F7E8093E2008091E2008160809319
:103CE000E2008091EC02882311F084E007C080910B
:103CF000E30087FD02C081E001C083E08093F00211
:103D00000E94511A8091E10083FF29C08091E20056
:103D100083FF25C08091E100877F8093E10082E0EE
:103D20008093F0021092EC028091E1008E7F8093EC
:103D3000E1008091E2008E7F8093E2008091E200BA
:103D400080618093E20042E060E080E00E94EC1C31
:103D50008091F00088608093F0000E94471AFF91E4
:103D6000EF91BF91AF919F918F917F916F915F91F3
:103D70004F913F912F910F900FBE0F901F9018956C
:103D80001F920F920FB60F9211242F933F934F93D0
:103D90005F936F937F938F939F93AF93BF93CF93D3
:103DA000DF93EF93FF93C091E900CF708091EC0017
:103DB000D82FD17080FDD0E81092E9008091F000FA
:103DC000877F8093F00078940E94041F1092E9008E
:103DD0008091F00088608093F000CD2BCF70C0936D
:103DE000E900FF91EF91DF91CF91BF91AF919F914A
:103DF0008F917F916F915F914F913F912F910F9094
:103E00000FBE0F901F9018951F93CF93DF93CDB7E0
:103E1000DEB7AA970FB6F894DEBF0FBECDBFE1EFB5
:103E2000F2E08091F100819322E0E93FF207C9F7C7
:103E30000E946F1A8091E80083FF2EC18091F102E9
:103E40009091F202492F50E04A30510508F024C108
:103E5000FA01E759FF4F0C949420803821F0823802
:103E600009F01AC108C08091ED029091EE029923E9
:103E700089F082600FC08091F5028F70873008F062
:103E80000BC18093E9008091EB0085FB882780F9C6
:103E90001092E9009091E800977F9093E80080935A
:103EA000F1001092F100D1C0282F2D7F09F0F4C04D
:103EB000882319F0823061F0EFC08091F3028130E5
:103EC00009F0EAC0933009F080E08093EE022EC042
:103ED0008091F30281112AC08091F5028F702FEF3B
:103EE000280F263008F0D8C08093E9002091EB001D
:103EF00020FF1CC0933021F48091EB00806214C03D
:103F00009091EB0090619093EB0021E030E0A901EB
:103F100002C0440F551F8A95E2F74093EA001092C1
:103F2000EA008091EB0088608093EB001092E9003A
:103F30008091E800877F8093E8000E94211DACC03B
:103F40008111AAC01091F3021F778091E30080785D
:103F5000812B8093E3008091E800877F8093E800C5
:103F60000E94211D8091E80080FFFCCF8091E3003A
:103F700080688093E300111102C082E001C083E0F9
:103F80008093F00289C08058823008F085C080910B
:103F9000F3029091F4028C3D53E0950779F583E0AC
:103FA0008A838AE289834FB7F894DE01139620E072
:103FB0003EE051E2E32FF0E050935700E49120FF00
:103FC00003C0E295EF703F5FEF708E2F90E0EA3014
:103FD00010F0C79601C0C0968D939D932F5F24313A
:103FE00049F74FBF8091E800877F8093E8006AE23D
:103FF00070E0CE0101960E942D1C16C06091F50262
:104000007091F602AE014F5F5F4F0E94711BBC01C1
:10401000892B09F441C09091E800977F9093E800C4
:1040200089819A810E948B1C8091E8008B77809314
:10403000E80032C0803881F58091E800877F809366
:10404000E8008091EC028093F1008091E8008E7787
:1040500072CF811121C08091F3029091F4029927CF
:104060000297D4F48091E800877F8093E8008091E4
:10407000F3028093EC020E94211D8091EC028111D9
:1040800006C08091E30087FD02C081E001C084E0AA
:104090008093F0020E945B1A8091E80083FF0AC0BF
:1040A0008091E800877F8093E8008091EB00806238
:1040B0008093EB00AA960FB6F894DEBF0FBECDBF7B
:1040C000DF91CF911F9108950895CF938091F002D1
:1040D0008823A1F0C091E900CF709091EC00892F66
:1040E000817090FD80E8C82B1092E9008091E80073
:1040F00083FD0E94041FCF70C093E900CF91089503
:1041000097FB072E16F4009407D077FD09D00E9484
:104110009A2007FC05D03EF4909581959F4F089515
:10412000709561957F4F0895EE0FFF1F0590F491F4
:10413000E02D0994AA1BBB1B51E107C0AA1FBB1F9E
:10414000A617B70710F0A61BB70B881F991F5A9523
:10415000A9F780959095BC01CD010895FB01DC0184
:1041600004C08D910190801921F441505040C8F74E
:10417000881B990B0895F999FECF92BD81BDF89ADD
:10418000992780B50895A8E1B0E042E050E00C9492
:10419000EF20262FF999FECF92BD81BDF89A0197A5
:1041A00000B4021639F01FBA20BD0FB6F894FA9A7F
:1041B000F99A0FBE08950396272F0E94CA200E94E5
:1041C000C920252F0E94CA20242F0C94CA200196B2
:1041D000272F0E94CA200C94C920DC01CB01FC01CE
:1041E000F999FECF06C0F2BDE1BDF89A319600B450
:0E41F0000D9241505040B8F70895F894FFCF5B
:1041FE00C8004902280850011E0A14019F19C2194D
:10420E00A319321A2E1AA21901E200E900EA00B52A
:10421E0000B600B700CD008301CC008A0192019454
:10422E00012102230224022502260227022A02B3BA
:10423E0000B4006F007000818283E200E900EA00A2
:10424E00B500B600B700CD008301CC008A01920103
:10425E0094012102230224022502260227022A02A9
:0C426E00B300B4006F0070008182830078
:00000001FF
